:020000040000FA
:040000008A01052844
:08000800572883129813831698
:1000100007309C009D019B0186018501073081000E
:100020008312850186013D3081000530A6008B17C3
:100030008B16A201A301A401A901A5014220250854
:100040002A20860046204A20A50A2508033C031DD5
:100050001F281D2882072E283128342824083728F5
:1000600008002308372808002208372808008207DC
:100070007E340C34B6349E34CC34DA34FA340E3454
:10008000FE34CE3485145220851008000515522008
:10009000051108002330A000A100A10B4D28A00BE2
:1000A0004C280800FA30A100A10B54280800A70032
:1000B000030EA8003D308100A60B8328291879285B
:1000C000A20A2208093C031D812829148128A918A5
:1000D0007C28A30A2308093C031D8128A914812830
:1000E00029197F28A40A2408093C031D8128291501
:1000F0008128A20129106728A301A9107028A40152
:1001000029110530A600280E8300A70E270E0B111B
:020110000900E4
:00000001FF
